:020000040000FA
:04000000CB303A289F
:08000800A000030EA100831209
:100010008B1C32288B1031181428B11C3228643004
:10002000010203183128182800001628172818285C
:1000300019281A281B281C281D281E281F283110A3
:10004000B114A810031005190314AA0DA90DA80DC9
:10005000B00B322831152A08AF002908AE00280855
:10006000AD00B11081010B11210E8300A00E200EF6
:02007000090085
:0C007400203084008001840A80300402E7
:10008000031C3C281230B000F02183160C3085058B
:1000900087018312850187010730990000309A009B
:1000A000103083168E008312603083168F00831207
:1000B0000030831691009F008312C83083168100A0
:1000C000831231309000003083168C008312103080
:1000D0008B00831600309B001C141A088312BC008E
:1000E000851DEE22831610309B001C141A08831203
:1000F000BD00831630309B001C141A088312DE00EA
:10010000D52281018E018F010B118B100B108C01F8
:100110008B1798203119AE20B30B96280310851940
:100120000314B90DF030390203195421142389281E
:100130006400311808000B1D08000B11B1103114B8
:100140001230B000051DA928321483160113831242
:100150000800321083160117831208003111013094
:10016000B7008B132030370783169B001C141A0826
:100170008312A400A500C030A506103037078316EF
:100180009B001C141A088312A30000303707831643
:100190009B001C141A088312A2008B17321CD6284D
:1001A00022090339A200A309A409A50922082D02E6
:1001B000031D4E2923082E02031D4E2924082F0259
:1001C000031D4E2901303702031DEB283D18EB2893
:1001D0003D143E14FD2102303702031DF428BD18E2
:1001E000F428BD143E14092203303702031DFD28F4
:1001F0003D19FD283D153E14152204303702031D1C
:100200000629BD190629BD153E14212205303702E5
:10021000031D0F293D1A0F293D163E142D220630CD
:100220003702031D1829BD1A1829BD163E143C2299
:1002300007303702031D21293D1B21293D173E149C
:100240004E2208303702031D2A29BD1B2A29BD175B
:100250003E14592209303702031D33295E18332911
:100260005E143E1464220A303702031D3C29DE1856
:100270003C29DE143E146F220B303702031D452942
:100280005E1945295E153E147A220C303702031D93
:100290004E29DE194E29DE153E148822B70A0D308C
:1002A000370203180800B1280130B600B300B400CB
:1002B000B500B70085018701B1139820B30B9C29C5
:1002C000031085190314B90DF03039020319C3293D
:1002D000B40B9C29013037020319992202303702EE
:1002E00003199E22033037020319A3220430370278
:1002F0000319A822053037020319AD220630370250
:100300000319B222073037020319B7220830370227
:100310000319BC22093037020319C1220A303702FF
:100320000319C6220B3037020319CB220C303702D7
:100330000319D0229630B400311D5D293111321CD1
:10034000A6292D090339AD00AE09AF092F1CB11341
:100350002F1C5D29B11B5D292E185D29B1178B1348
:1003600020303707BB002F08BA00DB2110303707D9
:10037000BB002E08BA00DB2100303707BB002D0878
:10038000BA00DB218B1785018701B70AB6010D3052
:100390003702031C5D29D52208003E1C08003E10D0
:1003A0001030BB003D08BA00DB213030BB005E08D6
:1003B000BA00DB2108008B133A0883161C159A003B
:1003C00083123B0883169B0055309D00AA309D0088
:1003D0009C1464009C18E9291C1183128B170800D7
:1003E000FF30C800CA15CB15CC15CD15CE15CF15CD
:1003F000D015D115D215D3150800C130BD05FF3079
:10040000DE050130C405C0000030C200C6005F1028
:100410000800C230BD05FF30DE050230C405C00053
:100420000030C200C6005F100800C430BD05FF30B8
:10043000DE050630C405C0000030C200C6005F10F3
:100440000800C830BD05FF30DE050A30C405C00015
:100450000030C200C6005F100800D030BD05FF307C
:10046000DE053C181030BC181130C405C000003047
:10047000C200C6005F100800E030BD05FF30DE0599
:100480003C181830BC181930C405C0001830C20020
:10049000C6005F105F17C411441208007F30BD050D
:1004A000C030DE050830C505C1000030C300C700FC
:1004B0000800BF30BD05C030DE051030C505C100E5
:1004C0000030C300C70008003F30BD05C130DE0565
:1004D0003030C505C1000030C300C70008003F3000
:1004E000BD05C230DE055030C505C1000030C30077
:1004F000C70008003F30BD05C430DE053C18803021
:10050000BC188830C505C1000030C300C700080012
:100510003F30BD05C830DE053C18C030BC18C830BF
:10052000C505C100C030C300C700DF174513C513A0
:100530000800103085060030870608002030850648
:100540000030870608002130850600308706080045
:10055000223085060030870608000030850602300C
:100560008706080002308506023087060800003042
:1005700085060430870608000030850601308706AE
:100580000800003085062130870608000030850607
:1005900011308706080000308506083087060800FD
:1005A000003085061830870608003D18FD21BD186B
:1005B00009223D191522BD1921223D1A2D22BD1AED
:1005C0003C223D1B4E22BD1B59225E186422DE18C0
:1005D0006F225E197A22DE1988220800B601B30163
:1005E000B4013C1CF62ABC01BC14F82ABC013C1422
:1005F0003C08B6006400FC2AFD2AFE2AFF2A002BD4
:10060000FF30B41B8500B41F8501B30BFA2AB40B6D
:10061000FA2A0310B60CB608031DFA2A0030BB00F4
:100620003C08BA00DB2108008F08031908008F017D
:1006300078308E00C80F3E2DC80A441C442B461C3F
:10064000352BCA1C262BCA014A15522B4A1D2B2BAF
:10065000CA01CA15522BCA1D302BCA014A16522B89
:100660004A1E522BCA01CA14522B4A1D3A2BCA01E8
:100670004A16522BCA1D3F2BCA014A16522B4A1E3C
:10068000522BCA01CA14522BCA1C492BCA014A1543
:10069000522B4A1D4E2BCA01CA15522B4A1E522BF1
:1006A000CA014A15C41C792BC61C6A2BCB1C5B2BB8
:1006B000CB014B15872B4B1D602BCB01CB15872B0B
:1006C000CB1D652BCB014B16872B4B1E872BCB01EC
:1006D000CB14872B4B1D6F2BCB014B16872BCB1DC0
:1006E000742BCB014B16872B4B1E872BCB01CB14C6
:1006F000872BCB1C7E2BCB014B15872B4B1D832BC4
:10070000CB01CB15872B4B1E872BCB014B15441DE3
:10071000AE2B461D9F2BCC1C902BCC014C15BC2B1B
:100720004C1D952BCC01CC15BC2BCC1D9A2BCC0190
:100730004C16BC2B4C1EBC2BCC01CC14BC2B4C1D22
:10074000A42BCC014C16BC2BCC1DA92BCC014C16D8
:10075000BC2B4C1EBC2BCC01CC14BC2BCC1CB32B07
:10076000CC014C15BC2B4C1DB82BCC01CC15BC2B93
:100770004C1EBC2BCC014C15C41DE42BC61DD52B27
:10078000CD1CC62BCD014D155F13F22B4D1DCB2B70
:10079000CD01CD15F22BCD1DD02BCD014D16F22B59
:1007A0004D1EF22BCD01CD14F22B4D1DDA2BCD01B8
:1007B0004D16F22BCD1DDF2BCD014D16F22B4D1E0C
:1007C000F22BCD01CD14F22BCD1CE92BCD014D1513
:1007D000F22B4D1DEE2BCD01CD15F22B4D1EF22B24
:1007E000CD014D155F1B1B2C441E1B2C461E0C2CD3
:1007F000CE1CFD2BCE014E15292C4E1D022CCE01F8
:10080000CE15292CCE1D072CCE014E16292C4E1E9E
:10081000292CCE01CE14292C4E1D112CCE014E16A2
:10082000292CCE1D162CCE014E16292C4E1E292CFD
:10083000CE01CE14292CCE1C202CCE014E15292CF5
:100840004E1D252CCE01CE15292C4E1E292CCE0155
:100850004E15C51D502CC71D412CCF1C322CCF016D
:100860004F155E2C4F1D372CCF01CF155E2CCF1DA1
:100870003C2CCF014F165E2C4F1E5E2CCF01CF14A7
:100880005E2C4F1D462CCF014F165E2CCF1D4B2CDE
:10089000CF014F165E2C4F1E5E2CCF01CF145E2C65
:1008A000CF1C552CCF014F155E2C4F1D5A2CCF015C
:1008B000CF155E2C4F1E5E2CCF014F15451E852C8B
:1008C000471E762CD01C672CD0015015932C501D40
:1008D0006C2CD001D015932CD01D712CD00150164A
:1008E000932C501E932CD001D014932C501D7B2C94
:1008F000D0015016932CD01D802CD0015016932C73
:10090000501E932CD001D014932CD01C8A2CD001D3
:100910005015932C501D8F2CD001D015932C501EA8
:10092000932CD0015015C51EBA2CC71EAB2CD11C60
:100930009C2CD1015115C82C511DA12CD101D115D0
:10094000C82CD11DA62CD1015116C82C511EC82C63
:10095000D101D114C82C511DB02CD1015116C82C75
:10096000D11DB52CD1015116C82C511EC82CD10156
:10097000D114C82CD11CBF2CD1015115C82C511D2C
:10098000C42CD101D115C82C511EC82CD101511530
:10099000451FF02C471FE12CD21CD22CD20152153E
:1009A000DF13FE2C521DD72CD201D215FE2CD21DE6
:1009B000DC2CD2015216FE2C521EFE2CD201D21477
:1009C000FE2C521DE62CD2015216FE2CD21DEB2C11
:1009D000D2015216FE2C521EFE2CD201D214FE2C35
:1009E000D21CF52CD2015215FE2C521DFA2CD2012C
:1009F000D215FE2C521EFE2CD2015215DF1B272DC4
:100A0000C51F272DC71F182DD31C092DD301531522
:100A1000352D531D0E2DD301D315352DD31D132D7B
:100A2000D3015316352D531E352DD301D314352D37
:100A3000531D1D2DD3015316352DD31D222DD3014A
:100A40005316352D531E352DD301D314352DD31CFC
:100A50002C2DD3015315352D531D312DD301D31515
:100A6000352D531E352DD3015315CD214008C4001B
:100A70004108C5005F18DF145F1CDF104808C9007B
:100A80000C304A05031D05120C304B05031D851261
:100A90000C304C05031D05100C304D05031D851051
:100AA0000C304E05031D87100C304F05031D071138
:100AB0000C305005031D07100C305105031D871223
:100AC0000C305205031D07120C305305031D87110E
:100AD00049080E020318982D12304A05031D051609
:100AE00012304B05031D851612304C05031D0514ED
:100AF00012304D05031D851412304E05031D871459
:100B000012304F05031D071512305005031D071441
:100B100012305105031D871612305205031D0716AA
:100B200012305305031D8715FF30480203190800D2
:100B30008F08031D0800982049080E02031C982DF9
:100B400018304A05031D051206304A05031D051617
:100B500018304B05031D851206304B05031D851605
:100B600018304C05031D051006304C05031D0514F7
:100B700018304D05031D851006304D05031D8514E5
:100B800018304E05031D871006304E05031D8714CF
:100B900018304F05031D071106304F05031D0715BB
:100BA00018305005031D071006305005031D0714AB
:100BB00018305105031D871206305105031D871695
:100BC00018305205031D071206305205031D071683
:100BD00018305305031D871106305305031D871573
:020BE00008000B
:084000000300030003000900A6
:02400E00CC33B1
:10420000010003000300030003000200020002009B
:104210000200000000000000000003000300FF0097
:10422000020000000000000000000000000000008C
:104230000000C000C000C000C000C000C000FF00FF
:10424000FF00C300F300CF00FF00C300F300CF0066
:10425000FF00C300F300CF00FF00C300F300FF0026
:104260000100FF00FF00FF00FF00FF00FF00FF0054
:10427000FF00FF00FF00FF00FF00FF00FF00FF0046
:10428000FF00FF00FF00FF00FF00FF00FF00FF0036
:10429000FF00FF00FF00FF00FF00FF00FF00FF0026
:1042A000FF00FF00FF00FF00FF00FF00FF00FF0016
:1042B000FF00FF00FF00FF00FF00FF00FF00FF0006
:1042C000FF00FF00FF00FF00FF00FF00FF00FF00F6
:1042D000FF00FF00FF00FF00FF00FF00FF00FF00E6
:1042E000FF00FF00FF00FF00FF00FF00FF00FF00D6
:1042F000FF00FF00FF00FF00FF00FF00FF00AA001B
:00000001FF
